:020000040000FA
:06000000713001303A28C6
:08000800A000030EA100831209
:1000100005191028831601178312B23081002B288E
:1000200083160113831203140B190310A80DA90DD5
:10003000AA0DAB0DAC0DAC16FF302C02031D2B2806
:10004000FA302B02031D2B2831152A08AF0029088E
:10005000AE002808AD008B100B11210E8300A00EFE
:04006000200E090065
:0C007400203084008001840A80300402E7
:10008000031C3C281230B000562183160C30850525
:1000900087018312850187010730990000309A009B
:1000A000103083168E008312603083168F00831207
:1000B0000030831691009F008312C83083168100A0
:1000C000831231309000003083168C008312103080
:1000D0008B00BC1B6D28851D9621932181018E010B
:1000E0008F010B118B100B108C018B17862031198F
:1000F00089203821B30B8428031085190314B90D06
:10010000F03039020319E120C02176286400321052
:10011000080031110130B7008B13203037078316E8
:100120009B001C141A088312A40010303707831692
:100130009B001C141A088312A300A6000230A60616
:100140000030370783169B001C141A088312A20084
:10015000A7000130A7068B17321CB42822090339E7
:10016000A200A309A409A50924082F02031DDB2866
:1001700023082E02031DC92822082D02031DDB2897
:1001800001303702031DC9283D18C9283D143E140B
:10019000822126082E02031DDB2827082D02031DBD
:1001A000DB2801303702031DDA283D1CDA283D1018
:1001B0003E148C21DB28B70A0230370203180800EE
:1001C0008C280130B600B300B400B500B70085013B
:1001D0008701B1138620B30B072903108519031477
:1001E000B90DF030390203192E29B41F8501B41F4F
:1001F0008701B40B07293708B6080319B60003199D
:100200000529FF3085008700B6039630B400311D04
:10021000EA283111321C11292D090339AD00AE092C
:10022000AF092F1CEA288E018F010C1CEA280C1044
:100230002E1EEA288B1320303707BB002F08BA0088
:10024000412110303707BB002E08BA004121003091
:100250003707BB002D08BA0041218B1785018701A4
:10026000B70AB60102303702031CEA2893210800BE
:100270003E1C08003E101030BB003D08BA00412172
:1002800008008B133A0883161C159A0083123B084A
:1002900083169B0055309D00AA309D009C1464007D
:1002A0009C184F291C1183128B17080083160030ED
:1002B0009B001C141A088312BC00831610309B008C
:1002C0001C141A088312BD00831620309B001C14D6
:1002D0001A088312C3000130C3080319C300831630
:1002E00030309B001C141A088312C4004030D50023
:1002F0001030D6000430D7000130D8000230C100E1
:10030000C20008000130BD000130C100C200C800B9
:100310005414D410541108000130C100C20054100C
:10032000D410541508003D1882210800B601B3010D
:10033000B4013C1C9E29BC01BC14A029BC013C1486
:100340003C08B6006400A429A529A629A729A82944
:10035000FF30B41B8500B41B8700B41F8501B41F98
:100360008701B30BA229B40BA2290310B60CB6085F
:10037000031DA2290030BB003C08BA00412108003F
:1003800007305405031908008F08031908008F016E
:1003900078308E005D095B05CA005E095C05CB0004
:1003A0005B095D05CC005C095E05CD00C80803193A
:1003B000DF29FF303C1CC800C80FAB2A2023C20B2A
:1003C00008006430C200C10B08004308C1000130BE
:1003D000C800C9005508DF000E23D5005608DF000D
:1003E0000E23D6005708DF00551C0E23D7005808EF
:1003F000DF00D51C0E23D800551C022A571C5B14A5
:10040000D71C5B10551D082A571DDB14D71DDB10A8
:10041000D51D0E2A571E5B15D71E5B11551E142ABB
:10042000571FDB15D71FDB11D51E1A2A581C5B1668
:10043000D81C5B12551F202A581DDB16D81DDB1255
:10044000D51F262A581E5B17D81E5B13561C2C2A54
:10045000581FDB17D81FDB13D61C322A561F5C141B
:10046000D61F5C105418DC14D418DC145419DC109A
:10047000541D3E2ACE0B3E2ADB01DB01C5015B1871
:10048000C50ADB18C50A5B19C50ADB19C50A5B1A60
:10049000C50ADB1AC50A5B1BC50ADB1BC50A5C184B
:1004A000C50AC6015D18C60ADD18C60A5D19C60A66
:1004B000DD19C60A5D1AC60ADD1AC60A5D1BC60A20
:1004C000DD1BC60A5E18C60AC7015B085D06C000D0
:1004D0004018C70AC018C70A4019C70AC019C70A76
:1004E000401AC70AC01AC70A401BC70AC01BC70A5E
:1004F0005C085E06C0004018C70AC018C70AC70BD0
:10050000A02A5418882AD418942A5419992A080021
:10051000440845020318912A46084502031CA02AF4
:1005200008005410D414080044084502031CA02AF3
:10053000080045084602031CA02A1430CE0008001B
:100540005D08DB005E08DC005419DC105418DC1474
:10055000D418DC1408004808C9004A180516CA183F
:1005600085164A190514CA1985144A1A8714CA1A15
:1005700007154A1B0714CA1B87164B180716CB18FA
:10058000871549080E020318DD2A4C180512CC18ED
:1005900085124C190510CC1985104C1A8710CC1AED
:1005A00007114C1B0710CC1B87124D180712CD18D2
:1005B0008711FF304802031908008F08031D080047
:1005C000862049080E02031CDD2A4A180512CA18A3
:1005D00085124A190510CA1985104A1A8710CA1AB5
:1005E00007114A1B0710CA1B87124B180712CB189A
:1005F00087114C180516CC1885164C190514CC1902
:1006000085144C1A8714CC1A07154C1B0714CC1BE5
:1006100087164D180716CD1887150800C001DF088A
:100620000319DF035F184014DF1A40144008C001AB
:100630005F1C4014DF1E4014C005C00C5F0C080096
:100640004A180516CA1885164A190514CA198514B8
:100650004A1A8714CA1A07154A1B0714CA1B871699
:100660004B180716CB188715CA01CB014C18051279
:10067000CC1885124C190510CC1985104C1A87100E
:10068000CC1A07114C1B0710CC1B87124D180712F0
:10069000CD188711CC01CD015B08DD005C08DE00C0
:1006A000DB08031D0800DC08031D080054110800C6
:084000000E000300060002009F
:02400E00CC33B1
:10420000010078007A007C007E007B0079007F004E
:104210007D007A0078007E007C00FF00FF00FF0038
:104220000000F200F600FA00FE00F200F600FA00CC
:10423000FE00F200F600FA00FE00FF00FF00FF00A3
:10424000300005000500050005000900090009000F
:1042500009000D000D000D000D00FF00FF00FF0024
:104260000500FF00FF00FF00FF00FF00FF00FF0050
:10427000FF00FF00FF00FF00FF00FF00FF00FF0046
:10428000FF00FF00FF00FF00FF00FF00FF00FF0036
:10429000FF00FF00FF00FF00FF00FF00FF00FF0026
:1042A000FF00FF00FF00FF00FF00FF00FF00FF0016
:1042B000FF00FF00FF00FF00FF00FF00FF00FF0006
:1042C000FF00FF00FF00FF00FF00FF00FF00FF00F6
:1042D000FF00FF00FF00FF00FF00FF00FF00FF00E6
:1042E000FF00FF00FF00FF00FF00FF00FF00FF00D6
:1042F000FF00FF00FF00FF00FF00FF00FF00DD00E8
:00000001FF
